:10000000C720013A8800081BA7210B1DFC2A8B166C
:10001000903065210A0808396521F0308A051B30C7
:100020008400840A94218000841E11280A30AF00C5
:100030002F08463E2B201D0603192128AF0B182838
:1000400008282F08073C031C29281D08A008031DA9
:1000500065212F08503E82003F3467342F3400342E
:10006000113414340034033468340034153400344B
:10007000043410340234CA34C72008183034203411
:1000800000348F34043414343434033401340234EF
:100090000434B834A434C03406342434AC34883442
:1000A00026346028B629692802293A2900297128AE
:1000B0005C2819296E300928AC3065211E08AE0075
:1000C000A003A01B08289421403A9E1C03198A15FE
:1000D00060282E08622120036521A003031D6C28DF
:1000E0009B289421AC001130AC0203187A28A00B95
:1000F0007128082894212A1EAC15AA1EAC170739AE
:10010000AD00013EAE0020189421AE198F289D202D
:1001100089002D0889072C088800A5219B282C0818
:10012000413988003F3089000B1E9B28A7219B285E
:100130008C0A0C1E08288A150828EB30AE00063001
:10014000AF002F08413E2B201E190D061E1D010673
:100150000319B6280730AE07AF0BA1280108343ABF
:10016000031DD828002801088D00003403302F0219
:100170000318C528AF03AF0D8B192F14DD20AF0076
:1001800023302F078B181C3008002E0808003F3042
:10019000890083160814831208080800942194210A
:1001A0000F398D009421F0398D068C039D2008288D
:1001B000010E023E0639AF00AF0C2F08AF0DAF0D98
:1001C000AF0D2F02080062212B3062210C0E0F3878
:1001D00062213F30B729E73419345B347C3447342B
:1001E000F43466347034BF346E3451349F34B834D0
:1001F000A6340C34C0347434D934FF34C434BD3420
:100200003930B7299E1898281E19CE281E080319C0
:100210008C0108289D20890021308400C920891F75
:10022000132909082B208000890A840A841D0E29BD
:10023000080004308B050B169F190B171F188B1520
:100240000D088100043A03199F039F1D8B140A2196
:100250001A308E21F121083089001430C221F12199
:100260000A30A0008F210C081404F039031D052862
:100270000B110828201E4929EA3062211030622122
:100280000C30840000086521840AA00B4229B320A9
:100290000828C7200C08413E2B20AD00003008186C
:1002A000E3282D1CAD18473062212D080F392D1C75
:1002B000AD18503EAD19283062212D080F3862214B
:1002C0003F30B729A00365297730AC002C08AA007D
:1002D0000830A8005B30B221861F6C297F30660091
:1002E0008613B121AB012A09AB06AA1B8613AA1FEC
:1002F0008617AA0D1A30B221A80B7329AB1B8613DF
:10030000AB1F8617B121AB00FF306600C920861FE6
:10031000A917AB0B8729A91B66290834A0029321D2
:10032000A00B8F2908006421861B94292A30B22152
:10033000A8000314861F0310AA0DB121A80B992948
:10034000AA0C2830B2212A0908008B1E0800831647
:10035000081555308900AA30890088148818AE29FC
:1003600083121B30A900A90BB329093435300B15B2
:10037000AD00A003A01B08282D082B202D1FAD0ABF
:100380006521B929C421C5298400C621C7210008D7
:100390008800090884020808800009088407840A84
:1003A000080001300B1F1B3088000310A419031430
:1003B000A411A70DA60DA50DA40DA30DA20DA10DB1
:1003C00003182416880BD52908008800880C080C0F
:1003D0000006840A3F3909042B2088004030890731
:1003E00008001830840093218000840A841EF329B9
:1003F0000B1B052A183095008317BB22950A951E02
:10040000FD29103089002830C2211030A0000B1FB8
:10041000201E0B2A152AD12120030319152A0D3C71
:10042000031C152A063A031DD1218A140A1028300C
:100430009400CB30970006309600970A17082B20BF
:1004400095000739203E8400950DF030950503187E
:10045000950E150803100005031D031414088400ED
:10046000800D960B1D2A00138013940A94191B2AE1
:100470009401950197010A148901283084001F0C0A
:100480001C0CE521881995170819961788189614D9
:10049000081897141D0D1C0DE821881995150819C9
:1004A000171688181417081816171C0C1D0CE521B0
:1004B0008819161408191514881817150818141512
:1004C0001E0D1D0DE8218819171708191616881812
:1004D0001517081894171D0C1E0CE521881B141401
:1004E000081B1515881A9717081A94161F0D1E0D4C
:1004F000E821881B1416081B9715881A9516081AE8
:1005000096161E0C1F0CE521881B1714081B1516C8
:10051000881A1615081A94141C0D1F0DE821881B43
:100520009415081B9716881A9514081A961518081A
:100530009406190895061A0896061B0897060430B3
:1005400089001C30C421F83089001430C421A00B6C
:10055000072A0B1B1534D1211F3095008313BB22B2
:1005600004309506151DAF2A95031519AF2A1430CE
:1005700089002830C2292830960015088400831F7E
:10058000C42A800D800DC52A800C16088400800CBA
:10059000960A161EBD2A0800A234433412348B3446
:1005A0004134C13411340C349234A134C334223474
:1005B000933413340A340934243489348A3491341A
:1005C00014340B34C234213446340F349434C534DB
:1005D00096349734A4348D341734C63445348E346D
:1005E0000E34473495348F342534C734A63426343A
:1005F00027340D34C4348C34B121A0002C30B729F9
:100600002E34E034C434BF344D3427341134C43470
:1006100072344E34AF347234BB34DD346834113448
:1006200083345A345A3406343634FC34FC34AB3414
:10063000D534393409349534E0348334973468340C
:100640004434BF3421348C341E34C834B83472344A
:10065000AD341434D634E934723421348B34D73485
:10066000FF3465349C34FB34C934033457349E342E
:100670006334AA343A34403405345634E0343D34DB
:10068000CF34A3341134FD34A8344434FE34273439
:1006900096347F342B34C2346334983484345E34DB
:1006A00009346C34D73410343234D1344D34EA3414
:1006B000EC3406347034B93455343B34BA348534B0
:1006C00090344D34EE343834F7342A345B34C1344A
:1006D0002A34933484345F34CD34F4343134A23446
:1006E0007534BB340834E6344C341734A6347C34C7
:1006F00019346034D3340534B2348E346F34D93481
:100700004A34DD34B03407342934B034EE3479342B
:10071000F6344334033494348F341634D534AA3445
:100720003134E234CD3438349C3455347734CE34DB
:100730005B342C34A434FB3462348F341834613489
:100740001D3461344634BA34B434DD34D9348034A1
:10075000C83416343F3449347334A834E034773421
:10076000AB349434F1345F3462340E348C34F3346B
:100770000534EB345A3425349E3432342734CC34A7
:10078000D7341D342D34F8348E34DB34433485347F
:100790006034A634F6343F34B93470341A344334F8
:1007A000A134C4349234573438346234E534BC3420
:1007B0005B3401340C34EA34C4349E347F3429343D
:1007C0007A342334B6341F344934E0341034763468
:1007D0009C344A34CB34A134E7348D342D34D834AE
:1007E0000F34F9346134C434A3349534DE340B341B
:1007F000F5343C3432345734583462348434BE34A3
:084000000000000000000000B8
:02400E00F13F80
:10420000840066003000E400DA00FA0023002F008A
:10421000BD00CB00F000B200AD000C00AB00DB0035
:104220001600B200700070004F005C008B0011009F
:104230002F009900A8002C0073001300C6008A000C
:104240003500FD00E700ED00A300670046002500F3
:104250008D009800A500320019007A001200360087
:10426000250048006300C500B300DA00E300290020
:1042700000000000E0007C00FC00BA000100FF002C
:00000001FF
